:020000040000FA
:10000000000000308A00412817280F398207303459
:10001000313432343334343435343634373438349C
:100020003934413442344334443445344634F000A6
:10003000030EF1000A08F2008A010408F30083129B
:1000400003130C1C2728AB0A0319AC0A0C100B1D58
:1000500036280B11E008031D3028E1080319362863
:10006000E003600A0319E1030319E0088312031394
:100070007308840072088A00710E8300F00E700EFF
:10008000090008308A0000208A0187157E16DB27C8
:10009000081502222023E0240910861A4D2809148D
:1000A000861E5028A901AA0189100810EE267E118B
:1000B000B92703187E157E195E29F5260E30F42225
:1000C000FE1D65282A30FE1167282030FE152D22DE
:1000D000E2186C28621C56287E11B92703187E1579
:1000E0007E195E29A82700302E02031D7928803052
:1000F0002D02000003188C28FE1D81282330FE11DC
:1001000083282030FE150A30F5004030F6220A30F0
:10011000F5004F30F6226C28A908031D9A280A30F2
:10012000F5006130F622E321EC220A30F50085303B
:10013000F622F52632248F018E01AB01AC017E122E
:100140008B170910861AA2280230E100E830E0007F
:1001500044277E11B92703187E157E195E29E10810
:10016000031DA828E008031DA8280914861EB62828
:100170007E168B132A27DF08031D4B2926242C24E7
:100180000B30BA00EB30B900C230B8000030B70015
:100190002C08BF002B08BE000F08BD000E08BC00D5
:1001A0003C08B7023D08031C3D0FB8023E08031C83
:1001B0003E0FB9023F08031C3F0FBA02BA1F1729AE
:1001C000B709B809B70A0319B80A00303802031D85
:1001D000EB28643037020000031CF02887154B29F8
:1001E000871100303802031DF72814303702000051
:1001F0000318D12100303802031D00290F303702C7
:1002000000000318D12100303802031D09290A30EB
:10021000370200000318D12100303802031D1229D3
:100220000530370200000318D121D1214B290030BD
:100230003802031D1D29643037020000031C2229E7
:1002400087154B298711B70803194B29003038024D
:10025000031D2C291430370200000318D821003068
:100260003802031D35290F30370200000318D8214A
:1002700000303802031D3E290A30370200000318FF
:10028000D82100303802031D47290530370200000D
:100290000318D821D82100303802031D5129053018
:1002A00037020000031C5729081089105929081427
:1002B00089142C23A90A0319AA0A5628EC220A3009
:1002C000F5009730F622C02701305E02031D712928
:1002D0000B30F5009830F6220A30F500A930F622EE
:1002E000E42102305E02031DB2290A30F500BB3062
:1002F000F622DF0A04305F020319DF01DF08031D65
:100300009029DB272C2387110B30F5000330F622D0
:10031000E4210B30F5001530F622E021E0214128E0
:10032000871501305F02031D9B290A30F500CD308F
:10033000F6220130A80002305F02031DA5290A3011
:10034000F500DF30F6228030A80003305F02031D85
:10035000AF290A30F500F130F622FF30A800E32182
:100360007E114C2803305E02031DBE290B30F500C0
:100370003930F622F526E627E321412804305E02D3
:10038000031DCB290B30F5009830F6220B30F50019
:100390002730F622E4217E11DE01EC22A901AA0118
:1003A0004C28A80AA808031DD729FF30A800080078
:1003B000A803A808031DDE290130A8000800E021D9
:1003C000E421E421E421E421E721E721E721FA30D7
:1003D000F629C830F6296430F6293230F6290A3079
:1003E000F6290530F6290230F6290130A70004303D
:1003F000A6003D30A500A50BFB29A60BFB29A70BEA
:10040000F729080087120F30F6212030B9228030FA
:10041000B9220530F6212030B9228030B9220130CE
:10042000F6210630AF220C30AF221430AF224B221F
:10043000EC220930F500E630F6220930F500F830FC
:10044000F622E3210A30F5000A30F6220A30F500E0
:100450001C30F622E421EC220800A000C52220086E
:10046000881507128712F039B922200EF039B92AFF
:10047000A0000310A00DA00DA00DC522200840383B
:10048000AF220830A20058222D22F40A0319F50ADF
:10049000A20B432A08000230F5006F30F400083048
:1004A000A300A40124083822A40AA30B522A08009E
:1004B0008312031774088D0075088F0083160317C5
:1004C0008C178B138B1B612A0C14000000007E1EFE
:1004D0008B17831203170C088312031308000034D0
:1004E000003400341034103400340034003400344C
:1004F0000034003414341434003400340034003434
:100500000034003415341534003400340034003421
:10051000013401341534153401340134003400340D
:1005200010341034103410341034103400340034CB
:1005300014341434143414341434143400340034A3
:100540001534153415341534153415340034FF348E
:10055000FF34FF34FF34FF34FF34FF34FF34A00096
:10056000C5222008881107128712F039B922200EFF
:10057000F039081801388818023808190438881921
:100580000838880087168712080088178316031317
:10059000881783120313881107167E108716E62228
:1005A000881F7E148712E6228716E6228712E6222B
:1005B0007E1CCD2A8316031388138312031307129C
:1005C0000800000000000000000000000000000023
:1005D00000000000000008000130AF2A0230AF2AFE
:1005E0008030AF2AC030AF2A8038AF2A8312031779
:1005F0008D0075088F000323F4220323FF390319AC
:1006000008002D22FD2A831603178C178B138B1BD2
:10061000062B0C14000000007E1E8B17831203179C
:100620000C088D0A03198F0A831203130800203067
:100630002D2AA100210E05202D22210805202D2A7A
:100640008312031391010C30970083160313FF30BC
:100650009200071183120313280895000800373011
:1006600084000A30A2002F082202AF0030082202C4
:10067000B0003108A202FE10B0030319FE14B00A44
:10068000B008031D452B2C302D220008840AA3003E
:10069000AF08031D572BFE18542B30302302031DC7
:1006A000542B2030A300552BFE1423082D22AF0815
:1006B00003195B2BAF03B003A20B3C2B08003424BF
:1006C0002830A2003C30C3003230C400C101031006
:1006D000BA0CB90CB80CB70C031C872B0530A3005F
:1006E000430884000008C100440884004208C20195
:1006F0008007031C7D2B0130C20041088007031CCA
:10070000832B0130C200C30AC40AA30B702B031051
:10071000BC0DBD0DBE0DBF0DC00DA20B622B0800A0
:10072000A2013424BC08031DA22BBD08031DA22B6B
:10073000BE08031DA22BBF08031DA22BC008031D6A
:10074000A22B0800A20A0310C01BCA2BBC0DBD0DB2
:10075000BE0DBF0DC00D40083B02031DC02B3F085E
:100760003A02031DBF2B3E083902031DBE2B3D0874
:100770003802031DBD2B3C083702000000000000BA
:1007800000000318A22B34240310C00CBF0CBE0CB5
:10079000BD0CBC0C40083B02031DDF2B3F083A0296
:1007A000031DDE2B3E083902031DDD2B3D083802F8
:1007B000031DDC2B3C083702000000000000000095
:1007C000031CF42B3C08B7023D08031C3D0FB80284
:1007D0003E08031C3E0FB9023F08031C3F0FBA023C
:1007E0004008031C400FBB02B20DB30DB40DB50D94
:1007F000B60DA20BC42B080034242830A20005300B
:10080000A3003230840000080F39C10005304102D6
:10081000031C0C2C033080070008F039C100503055
:100820004102031C152C30308007840AA30B032CD3
:100830000310B70DB80DB90DBA0DBB0DB20DB30D48
:10084000B40DB50DB60DA20BFF2B0800B701B80112
:10085000B901BA01BB010800BC01BD01BE01BF0165
:10086000C001080026242C24B201B301B401B50153
:10087000B60108003308BD003208BC003408BE00D1
:100880003508BF003608C00008003308B800320839
:10089000B7003408B9003508BA003608BB000800B4
:1008A00026242C243730C3003630C4000530A20083
:1008B00044088400000E6424440884000008642472
:1008C000C403A20B582C08000F393038C10043086C
:1008D000840041088000C30A080034242830A300A3
:1008E0000310BB0CBA0CB90CB80CB70CB60CB50C99
:1008F000B40CB30CB20C373084000530A200801F5A
:10090000832C30308002801D872C03308002840AC3
:10091000A20B7F2CA30B702C080034243730C300AB
:100920003230C4000530A2004308840000080F39AB
:10093000A300840A000EF039A304440884002308AD
:100940008000C30AC30AC40AA20B942C452C831648
:1009500003178C18A92C7608831203178D007708CB
:100960008C00831603178C130C158B1355308D00D8
:10097000AA308D008C147E1E8B170C11831203136A
:1009800008008312031776088D00831603178C1353
:100990000C14831203170C0883120313080084003D
:1009A000C1248000840AF60AA20BD02C080084001F
:1009B0000008F700A724840AF60AA20BD82C080026
:1009C00083160317871583160313823099001811B5
:1009D0001812981683120313181698170800831616
:1009E00003132108200283120313031DF92C0310A3
:1009F000080083160313A00AE3302002031D022D12
:100A0000A230A00020088400000883120313FB001A
:100A1000031408000A30E8008C1E0C2D981C142DBD
:100A20001A08181218160C2D1A08FB001A2DEF219F
:100A3000E80B0C2D08000A2524307B02031D1B2D1A
:100A40000A2547307B02031D1B2D0A2550307B02EF
:100A5000031D1B2D0A2547307B02031D1B2D08009B
:100A60001B250A2553307B02031D302D0A254130FA
:100A70007B02031D302D83160317A130A0008312C3
:100A800003135030A3000A25831603178317200889
:100A900084002A307B020319552D7B088000A00AB0
:100AA000831203138313A30B432D831203138313A6
:100AB000080001309A263708D90002309A263708F4
:100AC000DA0033303702031D662DE214323037026C
:100AD000031D6B2D621408001B250A2547307B027D
:100AE000031D6C2D0A2541307B02031D6C2D8312E2
:100AF00003172130A000831203135030A3000A25EE
:100B0000831203178317200884007B0880002A3093
:100B10007B02031D8F2D831203138313952DA00ACF
:100B2000831203138313A30B7F2D08000230462684
:100B3000C7253808C6003708C5003908C7003A0875
:100B4000C80004304626C7253808CA003708C9003F
:100B50003908CB003A08CC00073046268D246D2496
:100B60003208D300083046268D246D243308D50082
:100B70003208D400093046268D246D243308D7006E
:100B80003208D60008308A006A208A0108008D24C5
:100B90006D2445243808E4003708E3003908E500EF
:100BA0003A08E6003B08E70009308A00CB218A01B9
:100BB0009023452409308A00CB218A015F23330822
:100BC000CE003208CD003408CF003508D0003608FA
:100BD000D1006408B8006308B7006508B90066086A
:100BE000BA006708BB004D08B7024E08031C4E0F41
:100BF000B8024F08031C4F0FB9025008031C500FD6
:100C0000BA025108031C510FBB022C240630BC0051
:100C1000902345242C240A30BC005F2345244D0832
:100C2000B7074E0803184E0FB8074F0803184F0FA9
:100C3000B90750080318500FBA0751080318510F8D
:100C4000BB0708004030F4223B0819233A08192357
:100C5000390819233808192337081923E3294030A4
:100C6000F42237082D2238082D2239082D223A087F
:100C70002D223B082D223C082D223D082D223E0826
:100C80002D223F082D2240082D22E329A200A20A8E
:100C900026242C24AF012030F9003730FA008312CB
:100CA00003178317F90A70307902031D5B2E831234
:100CB00003138313992E790884002A300002031D40
:100CC000652E8312031383136E2E2C3000028312C1
:100CD00003138313031D4F2EA20B4F2E83120317F2
:100CE0008317F90320307902031D7A2E8312031330
:100CF0008313992E790884002C3000028312031389
:100D000083130319992E8312031783170008F70022
:100D10008312031383132E30770203196E2E7A0881
:100D2000840077088000FA0AAF0A41307A02031D76
:100D30006E2E0800A200A20A26242C24AF01A030A7
:100D4000F9003730FA00831603178317F90AF030D9
:100D50007902031DAF2E831203138313ED2E79083E
:100D600084002A300002031DB92E8312031383135B
:100D7000C22E2C300002831203138313031DA32EF3
:100D8000A20BA32E831603178317F903A030790251
:100D9000031DCE2E831203138313ED2E79088400D6
:100DA0002C3000028312031383130319ED2E8316D4
:100DB000031783170008F7008312031383132E30E1
:100DC00077020319C22E7A08840077088000FA0A95
:100DD000AF0A41307A02031DC22E0800D301E2019E
:100DE00030256C255925962508006E27E218032F1B
:100DF0006218032F0A30F5002E30F6220A30F50073
:100E00008030F62208000A30F5007D30F6223224C8
:100E10005308B7000230AF00B001B1016B270A30B0
:100E2000F5007330F62232242808B7000330AF00F3
:100E3000B001B1016B27172348302D22172332242C
:100E40005508B8005408B7000330AF000230B000B6
:100E5000B1016B2F0030F42232242C08BA002B0889
:100E6000B9000F08B8000E08B7000530BC005F23BA
:100E700045240A30AF000230B000B1016B27483082
:100E80002D227A302D22172B0E30F42232246108C5
:100E9000B8006008B7002530BC0090233208DB00A2
:100EA0005C085B0203196A2F5B08DC0034245B08D2
:100EB000B7000230AF00B001B1016B2709305B020F
:100EC0000319732706305B020319942703305B0272
:100ED0000319F5260800FC2350242F2B0B30F500B6
:100EE0004B30F62208006E270B30F5005D30F622FD
:100EF0000630A2004D30840000082D22840AA20B87
:100F00007C2F08006E270B30F5006830F622322463
:100F10005708B8005608B7000530AF000130B000E0
:100F2000B1016B276D302D2A6E27621C9C2F0B3070
:100F3000F5006E30F6220800E21CA32F0B30F500FE
:100F40007B30F62208000B30F5008830F6220800CE
:100F50008530AB2F81309F00F5219F149F18AE2F55
:100F6000831603131E0883120313AD001E08AE0080
:100F7000080006080F390F3A03140319031008007C
:100F8000B927031CC02FDE0106080F39A400EF218A
:100F900006080F392402031DC32FDE0A241CD72F95
:100FA000DE0AA41CD72FDE0A241DD72FDE0AB9279C
:100FB0000318D72F0800F601C124A800FF3028022B
:100FC000031DE52F8030A800E62F0800F601280851
:100FD000F700A7240800FF3FFF3FFF3FFF3FFF3F11
:100FE000FF3FFF3FFF3FFF3FFF3FFF3FFF3FFF3F11
:100FF000FF3FFF3FFF3FFF3FFF3FFF3FFF3FFF3F01
:1010000083018312031789148316031368308F003A
:1010100007308100C33085002F3086008130870083
:10102000003088000030890080309F0000308E0042
:1010300001308C0000308D000F30950083160317AF
:1010400003308800003089008312031360308B0066
:10105000C33085002F308600813087000030880043
:101060000030890047309000063092002030840024
:1010700080016930040203193F28840A3828831646
:101080000313A230A100A0008312031308008A01F9
:10109000322408308A0008008A01262408308A0099
:1010A00008008A012C2408308A0008008A015F2386
:1010B00008308A0008008A01902308308A0008005E
:1010C0008A01452408308A0008008A013A24083041
:1010D0008A00080047204608B8004508B7004708BE
:1010E000B9004808BA004608E4004508E30047088C
:1010F000E5004808E600DC213C08B7073D08031876
:101100003D0FB8073E0803183E0FB9073F08031804
:101110003F0FBA0740080318400FBB073808C60046
:101120003708C5003908C7003A08C8005120983070
:10113000BE009630BD008030BC005B2060203708C8
:10114000CE004130CE0751209830BE009630BD0011
:101150008030BC00562065204C204608B800450869
:10116000B7004708B9004808BA003C08B7023D0874
:10117000031C3D0FB8023E08031C3E0FB9023F0896
:10118000031C3F0FBA024008031C400FBB02380883
:10119000C6003708C5003908C7003A08C800CB2187
:1011A0005B2060203708D0003030D007CB2156209C
:1011B00065204C204608B8004508B7004708B9002C
:1011C0004808BA003C08B7023D08031C3D0FB802AE
:1011D0003E08031C3E0FB9023F08031C3F0FBA0232
:1011E0004008031C400FBB0251201830BC005620A1
:1011F0006020CB215B2060203708D2004130D2072D
:101200006408C6006308C5006508C7006608C80012
:1012100047204A08B8004908B7004B08B9004C08F5
:10122000BA004A08E4004908E3004B08E5004C080E
:10123000E600D3213C08B7073D0803183D0FB80767
:101240003E0803183E0FB9073F0803183F0FBA07BF
:1012500040080318400FBB073808CA003708C90008
:101260003908CB003A08CC0051200130BF003130A2
:10127000BE002D30BD005B2060203708CD0041301E
:10128000CD0751200130BF003130BE002D30BD00F0
:10129000562065204C204A08B8004908B7004B0882
:1012A000B9004C08BA003C08B7023D08031C3D0FCA
:1012B000B8023E08031C3E0FB9023F08031C3F0F53
:1012C000BA024008031C400FBB023808CA003708A6
:1012D000C9003908CB003A08CC00CB213C08BC0738
:1012E0003D0803183D0FBD073E0803183E0FBE071B
:1012F0003F0803183F0FBF0740080318400FC007FF
:101300005B2060203708CF003030CF07CB213C086E
:10131000BC073D0803183D0FBD073E0803183E0FEC
:10132000BE073F0803183F0FBF0740080318400FD0
:10133000C007562065204C204A08B8004908B7006D
:101340004B08B9004C08BA003C08B7023D08031C22
:101350003D0FB8023E08031C3E0FB9023F08031CB4
:101360003F0FBA024008031C400FBB0251200C3053
:10137000BC0056206020CB215B2060203708D100C4
:101380004130D1076408CA006308C9006508CB0072
:101390006608CC00080051200F30BE004230BD006E
:1013A0004030BC00080051200A30BF00BA30BE00F7
:1013B0009530BD00BC01080051200530BF005D30F4
:1013C000BE004A30BD008030BC0008000034463406
:1013D000723465347134753465346E347A346E34F5
:1013E0006F3472346D3461346C3420342034003402
:1013F0004034313430344D3448347A34203420345D
:1014000028346334293444344C3434344A34413439
:101410004C3400340034563431342E3430343134CA
:10142000203420342034303432342E3430343234CA
:101430002E34313432340034403456346134723412
:10144000693461346E34743465342034313420347A
:1014500020342034203420342034003400345334F9
:10146000613474342D3453347534633468346534E2
:1014700021342034203420342034203420340034EB
:1014800040344134753466346834653469347A34B0
:1014900065346E3421342034203420340034003458
:1014A00054346834653472346D346F347334743446
:1014B0006134743420344C344F3457342034203465
:1014C0000034003454346834653472346D346F340D
:1014D000733474346134743420344F344B342034D6
:1014E000203420340034403450342034003440342C
:1014F000503457344D343A3400344D34533400347E
:101500004D3453342D342D340034003431342E34E2
:101510004D3465347334733475346E346734213428
:10152000203420342034203420342034003400345B
:10153000543461347334743465346E3465346934CE
:101540006E3467346134623465342034203420349E
:10155000003440345434613473347434653420348A
:1015600031342034203420342034203420342034CA
:1015700020342034003400344D34653473347334F3
:1015800075346E3467343A342034203420342034B7
:101590002034203420342034003440345034573444
:1015A0004D343D3431342034203420342034203440
:1015B000203420342034203420342034003440348B
:1015C000503457344D343D3431343234383420348F
:1015D000203420342034203420342034203420346B
:1015E00000344034503457344D343D343234353483
:1015F0003534203420342034203420342034203436
:1016000020342034003440344E346F3472346D341E
:1016100061346C347A3475347334743461346E34B8
:1016200064342034203420340034403431343034B5
:101630002034533465346B3420347734613472345D
:10164000743465346E342034203420340034403413
:101650005434613473347434653420343434203475
:1016600020342034203420342034203420342034DA
:101670000034003453347434613472347434773445
:1016800065347234743420344E3445345534203447
:1016900020342034003440342034203420342034AA
:1016A000203420342034203420342034203420349A
:1016B0002034203420342034003440344C346F340F
:1016C0006334613474346F3472343A342034003407
:1016D00040344E344E343A342034003440344E34A6
:1016E000613476342D344D346F34643465342034B1
:1016F00032344434003440344E34613476342D3442
:101700004D346F346434653420343334443400341D
:1017100040344E34613476342D344D346F34643477
:10172000653420345334753463346834653400349C
:1017300000346B34653469346E3465342034463497
:1017400075346E346B34743469346F346E340034F1
:10175000FF3FFF3FFF3FFF3FFF3FFF3FFF3FFF3F99
:10176000FF3FFF3FFF3FFF3FFF3FFF3FFF3FFF3F89
:10177000FF3FFF3FFF3FFF3FFF3FFF3FFF3FFF3F79
:10178000FF3FFF3FFF3FFF3FFF3FFF3FFF3FFF3F69
:020000040000FA
:020000040000FA
:04400E00D320FF3F7D
:020000040000FA
:08400000FF3FFF3FFF3FFF3FC0
:020000040000FA
:02401200FF3F6E
:00000001FF
